:1000000030C04AC049C148C047C046C005C370C1DE
:1000100043C042C041C086C53FC03EC03DC03CC099
:100020003BC04552520A00204F4B0A004552520A2B
:10003000004F4B0A00204F4B0A004F4B0A0045521D
:10004000520A004F4B0A004D454D20000A68656C6E
:100050006C6F20000A68656C6C6F20756172743279
:10006000200011241FBECFE5D2E0DEBFCDBF11E0DE
:10007000A0E6B0E0E8E9F3E102C005900D92A438F3
:10008000B107D9F722E0A4E8B1E001C01D92AD307C
:10009000B207E1F7BAD57EC9B3CF8091A301811130
:1000A00001C0C29A2091A30130E08091910190E0BB
:1000B000AC01440F551F440F551F840F951F880F27
:1000C000991F880F991F64E670E06AD826173707D2
:1000D00009F4C2988091A301843121F08F5F80934D
:1000E000A30108951092A301089580918F018823A0
:1000F00091F18091A20191E0980F9093A2018F71EC
:1001000051F59091900180919101891720F48F5FB2
:10011000809391010AC0981720F481508093910137
:1001200004C0981302C010928F01E0919101F0E099
:10013000E05AFF4F8081811104C080B78F7780BF64
:1001400003C080B7806880BFE0919101F0E0E05A81
:10015000FF4F808186BF08958091A10191E0980FA3
:100160009093A101837029F58091AE01882309F154
:1001700020919F013091A001A9014F5F5F4F5093E3
:10018000A00140939F01243F314048F480FF05C007
:100190009BB380E289278BBB0895DD980895DD9895
:1001A0001092A00110929F018091AE0186958093DC
:1001B000AE0108958091AD018823E1F31092AD0165
:1001C0008091AB0108958091AD0108959091AC01AB
:1001D0009111FCCF80958093A8018AE08093AC01B7
:1001E0000895CF93E7DFC82FF1DF8C2FCF910895CB
:1001F000CF93DF93EC018881882329F02196E6DFF5
:1002000089918111FCCFDF91CF910895CF93DF9336
:1002100090939E0180939D01FC012491222369F01B
:10022000EC01FE012196D0939E01C0939D01849123
:10023000CDDFFE0184918111F4CFDF91CF9108953C
:100240009B01AC01D69ADE9ADF9A60E874E88EE1F1
:1002500090E0B9D73093A7012093A601C9019695E4
:100260008795280F391F3093A5012093A4018CB5E1
:100270009DB501969BBD8ABD8EB582608EBD8FB542
:10028000806C8FBD619A979A8BB780618BBF1092FB
:10029000AC011092AD0108951F920F920FB60F920C
:1002A00011242F933F938F939F93F894CF9917C066
:1002B0002CB53DB58091A4019091A501820F931FAB
:1002C00099BD88BD1092A90181E08093AA015A9A34
:1002D000CF9904C08CB186608CB9979878949F911F
:1002E0008F913F912F910F900FBE0F901F901895F7
:1002F0001F920F920FB60F9211242F933F938F935B
:100300009F93EF93FF93F89499B38091AA01882368
:10031000C9F099233CF49091AA018091A901892BFD
:100320008093A9018091AA01880F8093AA0128B522
:1003300039B58091A6019091A701820F931F99BDB5
:1003400088BD27C081E08093AD018091A901809391
:10035000AB01E0918C01EE3150F481E08E0F80937F
:100360008C018091AB01F0E0E151FE4F80838091E0
:10037000AB018A3059F4E0918C01F0E0E151FE4F7D
:10038000108281E080938B0110928C01619A6298B7
:10039000979A7894FF91EF919F918F913F912F9130
:1003A0000F900FBE0F901F901895CF93DF93CFEA59
:1003B000D1E0FE0120E066E458E540E331E38991B5
:1003C0009991A991B991813072E0970773E0A707DD
:1003D000B10599F028F40397A340B10591F01AC034
:1003E0008330910571E0A70772E0B70761F08130B3
:1003F0009240A140B24019F00DC0608305C0408317
:1004000003C0308301C050832F5F31962C30B9F682
:100410008CE001C080E0DF91CF9108954091B00160
:10042000453009F468C020E030E090E080E051E021
:100430000BC0292F30E0F901E155FE4F41814530D5
:1004400009F456C091118F5FF901E155FE4F2081EB
:10045000211112C0413039F4E82FF0E0E155FE4F90
:1004600050839F5F41C0433009F042C0E82FF0E065
:10047000E155FE4F508338C0223089F4413039F4C1
:10048000E82FF0E0E155FE4F50839F5F2DC04330D1
:1004900079F5E82FF0E0E155FE4F508325C021307B
:1004A00089F4411107C0E82FF0E0E155FE4F1082BA
:1004B0009F5F1AC04230E1F4E82FF0E0E155FE4FB3
:1004C000108212C02330A1F4411107C0E82FF0E0E0
:1004D000E155FE4F10829F5F07C0423049F4E82F7C
:1004E000F0E0E155FE4F10829F5F903408F4A1CFF9
:1004F000803410F0089580E0982F27E0E92FF0E095
:10050000E155FE4F20839F5F9034C0F3089589B377
:1005100083FB882780F9982F80938701809186013B
:10052000981323C0809185018F5F8093850191117D
:1005300064C0853108F461C080918801813009F080
:100540005CC08091890190918A019C0129523109F6
:100550002E30310508F051C022E020938801FC01C3
:10056000E155FE4F25E0208348C0811150C08091A5
:100570008501853108F446C090918801911142C0EF
:1005800010928A011092890191E090938801853040
:1005900018F4109284010FC082E0809384010BC094
:1005A00080918501853020F481E08093840103C02F
:1005B00083E0809384018091890190918A01803445
:1005C000910570F4009731F020918401FC01E2550F
:1005D000FE4F2083019690938A01809389010BC07E
:1005E00010928801FC01E155FE4F25E02083109216
:1005F0008A01109289011092850180918701809370
:1006000086010895909188019130A9F7C0CF80911B
:100610008801813081F7C4CF1F920F920FB60F92DD
:1006200011242F933F934F935F936F937F938F93F7
:100630009F93AF93BF93EF93FF93F8942AB53BB585
:100640008091A6019091A701820F931F9BBD8ABD47
:100650008091AC018823D1F081508093AC01893026
:1006600089F08091A80180FD04C08FB580648FBDA2
:1006700003C08FB58F7B8FBD8091A8018695809335
:10068000A80106C08FB58F7B8FBD02C040DF2DDD76
:100690007894FF91EF91BF91AF919F918F917F914E
:1006A0006F915F914F913F912F910F900FBE0F90DF
:1006B0001F9018952F923F924F925F926F927F9268
:1006C0008F929F92AF92BF92CF92DF92EF92FF9262
:1006D0000F931F93CF93DF93CDB7DEB728970FB655
:1006E000F894DEBF0FBECDBF322E232E49835A832E
:1006F0006B837C838D839E83A9E0F5D509F008F494
:1007000081C044244394512C612C712C812C912C58
:1007100018861F82242D352D462D572D682D792DB5
:1007200088859F8101E0BDD5822E932E48875F8307
:10073000B62FA72FF82FE92F02E0B3D5A22EB32EA4
:10074000C42ED52EE62EF72E082F192F282D392D41
:1007500048855F816B2F7A2F8F2F9E2FBBD5422E1E
:10076000532E642E752E862E972E88879F83A22E59
:10077000B32EC42ED52EE62EF72E082F192F232D9B
:10078000322D49815A816B817C818D819E813FD53B
:10079000A9E0A9D511F008F0BDCFA42CB52CC62C2A
:1007A000D72CE82CF92C08851F81232D322D498167
:1007B0005A816B817C818D819E8129D50F2EFAE033
:1007C000AF2EF02DB12CC12CD12CE12CF12C00E05E
:1007D00010E01BD580E3820FF9DC242D352D462D4A
:1007E000572D682D792D88859F8111D5422E532E46
:1007F000642E752E862E972E88879F83A0E073D552
:1008000061F615C00F2EFAE0AF2EF02DB12CC12CE1
:10081000D12CE12CF12C00E010E049815A816B8150
:100820007C818D819E81F1D480E3820FCFDC28967C
:100830000FB6F894DEBF0FBECDBFDF91CF911F91F1
:100840000F91FF90EF90DF90CF90BF90AF909F906F
:100850008F907F906F905F904F903F902F90089572
:10086000CF92DF92EF92FF921F93CF93DF936B01B2
:100870007C01142F442301F1C1E0D0E0212F30E0AE
:1008800021503109CE01022E02C0880F991F0A940F
:10089000E2F7092E000CAA0BBB0B8C219D21AE2187
:1008A000BF2104C0B695A795979587952A95D2F74D
:1008B000805D8CDC115011F7DF91CF911F91FF907B
:1008C000EF90DF90CF900895FC012081222339F032
:1008D000319680E08F5F91919111FCCF089580E077
:1008E0000895CF92DF92EF92FF920F931F93CF93D1
:1008F000DF93D62FC82ED12CE12CF12C062F10E03F
:1009000001501109101611067CF4682F7D2D8E2DD3
:100910009F2DC0E0A70196010AD4CF5F2C2F30E0B5
:1009200020173107BCF304C0682F7D2D8E2D9F2D1D
:10093000D11104C061E070E080E090E0DF91CF91E0
:100940001F910F91FF90EF90DF90CF900895CF927D
:10095000DF92EF92FF920F931F93CF93DF93662363
:10096000B9F1FC01108120ED210F2A30A8F007C059
:100970001991015080ED810F8A30A8F003C0C12C7D
:10098000D12C7601C701B6012AE030E040E050E00A
:100990001AD469017A011FC00FEF060FEC012196EE
:1009A000C12CD12C7601602F8AE09BDF9B01AC012A
:1009B000812F110F990BC097BC01990F880B990BD0
:1009C000B6D3C60ED71EE81EF91E0111D1CF03C043
:1009D000C12CD12C7601C701B601DF91CF911F91B7
:1009E0000F91FF90EF90DF90CF9008950F931F939A
:1009F000CF93DF93FC01962F00E010E09801A1E077
:100A0000B0E027C0EF01C90FD11D4881403391F4F8
:100A1000AD01092E02C0440F551F0A94E2F740951C
:100A20005095052E000C660B770B04231523262307
:100A300037230FC0AD01092E02C0440F551F0A9481
:100A4000E2F7052E000C660B770B042B152B262BDB
:100A5000372B9150B8F6C901B801DF91CF911F91A2
:100A60000F910895FC012081222379F1319660E0F5
:100A700070E0CB01422F30ED320F3A3060F021565A
:100A8000263018F439EA340F06C02FEB240F263035
:100A9000F8F439EC340FDC01CB01880F991FAA1F41
:100AA000BB1F880F991FAA1FBB1F880F991FAA1F62
:100AB000BB1F880F991FAA1FBB1F3F70BC01CD0130
:100AC000632B21912111D6CF089560E070E0CB0116
:100AD0000895CF93DF9300D0CDB7DEB78823A1F080
:100AE0001A82198229813A812239334059F02981A9
:100AF0003A812F5F3F4F3A83298329813A812239F6
:100B00003340A9F7815061F70F900F90DF91CF919B
:100B1000089584E087BB83E080BF81E083BF89BF05
:100B200016BE08951F920F920FB60F9211242F93A5
:100B30003F934F935F938F939F93F89480919C0181
:100B400091E0980F90939C01837029F58091AE01FC
:100B5000882309F120919A0130919B01A9014F5FEF
:100B60005F4F50939B0140939A01243F314048F4DA
:100B700080FF05C09BB380E289278BBB0CC0DD984A
:100B80000AC0DD9810929B0110929A018091AE01EB
:100B900086958093AE0178949F918F915F914F914C
:100BA0003F912F910F900FBE0F901F901895809539
:100BB000DA98F8949AE0EFE9F1E03197F1F700C0A4
:100BC000000080FF02C0DA9801C0DA9A8695915041
:100BD00091F77894089590939901809398019C01DE
:100BE000FC014491442381F03196F0939901E09304
:100BF0009801F9018491DBDFE0919801F09199016E
:100C00009F0184918111F0CF0895CF93DF93CDB7E9
:100C1000DEB72B970FB6F894DEBF0FBECDBF04B77B
:100C200014BE9FE088E10FB6F894A89581BD0FBE71
:100C300091BDD59ABA9AD398DB98F89460E875E29A
:100C400080E090E0FDDA65DF7894D29A84E590E068
:100C5000C2DF10E3812FABDF1F5F1533D9F78CE4C0
:100C600090E0D4DA202F30E040E050E060E070E027
:100C700080E090E01FDD8AE0A9DA8AEA8093AE0185
:100C80008EE891E059D3813009F04FC087E490E0BD
:100C9000BDDA86E090E050D380939101E82FF0E038
:100CA000E05AFF4F8081882351F080B7806880BF71
:100CB000E0919101F0E0E05AFF4F808186BF2091E2
:100CC00091012093900130E040E050E060E070E05E
:100CD00080E090E0EFDC80E279DA0F2EF0E0EF2E9A
:100CE000F0E0FF2EF02D02E911E00F2EF8E9CF2EF3
:100CF000F1E0DF2EF02DC70127D3D8018D939D930E
:100D00008D01AC01242F352F40E050E060E070E011
:100D100080E090E0CFDC80E259DAB2E0EB0EF11C2B
:100D2000C016D10641F78AE051DA0F2EFDE0EF2E12
:100D3000F2E0FF2EF02D0F2EF8E9AF2EF1E0BF2EDE
:100D4000F02D0F2EF3E06F2EF02D0F2EFFEECF2E95
:100D5000F1E0DF2EF02D0F2EF5E07F2EF02D0F2E7F
:100D6000FBEB2F2EF1E03F2EF02DA89580918B010B
:100D7000882309F4B0C10FEE11E0F801DF01808192
:100D8000803211F08A3009F41C923196EE16FF067B
:100D9000A9F744E050E060E671E08FEE91E0AFD259
:100DA000892B09F4FFCF44E050E065E671E08FEE57
:100DB00091E0A5D2892B09F04FC06091910186E0A6
:100DC00090E0C7D22091910130E040E050E060E037
:100DD00070E080E090E06EDC80E2F8D90F2EF0E069
:100DE0008F2EF0E09F2EF02D0F2EF2E94F2EF1E026
:100DF0005F2EF02D5D824C82F201619171912F0185
:100E0000C401B5D2AC81BD814D915C91242F352FA9
:100E100040E050E060E070E080E090E04BDC80E299
:100E2000D5D9B2E08B0E911C4A145B0419F761E02E
:100E30008EE891E08ED286E090E07ED29091910192
:100E4000891305C083E490E0E1D9562C09C08EE3F4
:100E500090E0DCD9562C04C00F2EFEE15F2EF02D61
:100E600044E050E06AE671E08FEE91E048D2892BD1
:100E700041F52091910130E040E050E060E070E009
:100E800080E090E017DC80E2A1D90F2EF2E98F2EEE
:100E9000F1E09F2EF02DF401419151914F01242F4B
:100EA000352F40E050E060E070E080E090E002DC50
:100EB00080E28CD9A814B90471F78AE390E0A6D92E
:100EC000562C44E050E06FE671E08FEE91E017D2CF
:100ED000892B49F484EF91E0F7DC682F84EF91E0EF
:100EE00085DD6093AE0144E050E064E771E08FEE91
:100EF00091E005D2892BC1F484EF91E0E5DC682F05
:100F000084EF91E024DD262F6093900181E08093AF
:100F10008F0130E040E050E060E070E080E090E081
:100F2000C9DB85E390E072D944E050E069E771E005
:100F30008FEE91E0E4D1892B09F047C086EF91E074
:100F4000C3DC682F86EF91E002DD4B01683EF3E0E1
:100F50007F0760F561E084EF91E0F9DC660F771FB1
:100F6000FB01EE56FE4F80EE99E7B40105D1718387
:100F700060830F2EF2E98F2EF1E09F2EF02DD40129
:100F80004D915D914D01242F352F40E050E060E000
:100F900070E080E090E08EDB80E218D9A814B904FC
:100FA00071F781E390E032D9562C0FC0AB01282DA8
:100FB000352F40E050E060E070E080E090E07ADBC8
:100FC00080E204D98CE290E021D944E050E06EE761
:100FD00071E08FEE91E093D1892B09F074C086EF18
:100FE00091E072DC982E84EF91E03CDD862E880C37
:100FF000292D30E040E050E060E070E080E090E0DB
:1010000059DB80E2E3D8282D30E040E050E060E09A
:1010100070E080E090E04EDB80E2D8D886EF91E08F
:10102000E7D880E2D3D8A89519821A821B8250FC97
:1010300047C0981045C0992099F0812C682D70E028
:101040006A507E4F42E050E0CE01019666D1CE015B
:10105000019608DD862FABDD83948394891470F3A9
:101060008AE0A5DDA895992039F1812C682D70E0E2
:101070006A507E4F42E050E0CE0101964ED1CE0143
:101080000196F0DCAB01BC019A01AB0160E070E0BD
:10109000CB012C833D834E835F83688779878A8762
:1010A0009B8760E070E080E090E004DB80E28ED817
:1010B000839483948914D0F287E290E0A7D803C088
:1010C00082E290E0A3D8D8011D928D01EA16FB06BA
:1010D000D1F710928B01809188018230A9F465D9F3
:1010E0008C3011F50FEA11E0F80181918F016ED873
:1010F00020163106C9F78AE069D816C07192CE165B
:10110000DF06E1F71092880120918D01822F6AE0BD
:1011100027D0992321F02F5F20938D0102C01092D8
:101120008D0184E1D6DC21CEEFEAF1E0E7CFEE27B6
:10113000FF27AA27BB2708C0A20FB31FE41FF51F74
:10114000220F331F441F551F9695879577956795F6
:1011500098F37040A9F7009799F7BD01CF01089562
:10116000991B79E004C0991F961708F0961B881FF9
:101170007A95C9F780950895AA1BBB1B51E107C05A
:10118000AA1FBB1FA617B70710F0A61BB70B881F17
:10119000991F5A95A9F780959095BC01CD010895A6
:1011A00097FB072E16F4009406D077FD08D0E4DFF5
:1011B00007FC05D03EF4909581959F4F089570955A
:1011C00061957F4F0895A1E21A2EAA1BBB1BFD015A
:1011D0000DC0AA1FBB1FEE1FFF1FA217B307E40716
:1011E000F50720F0A21BB30BE40BF50B661F771F6E
:1011F000881F991F1A9469F760957095809590954E
:101200009B01AC01BD01CF010895689401C0E89431
:101210008F929F92CF93DF9305D0DF91CF919F90D4
:101220008F90089588249924F401E401B0E41B2EE2
:10123000D4019D158E049F04E007F10738F4FC01EA
:101240004B01CA01B901AD019E011694220F331F53
:10125000441F551F661F771F881F991F881C991CE4
:10126000EE1FFF1FCC1FDD1FAA1FBB1F8A149B048C
:10127000EC05FD05CE05DF05A007B10748F08A188B
:101280009B08EC09FD09CE09DF09A00BB10B216019
:101290001A94E1F62EF49401AF01BE01CD01000CC9
:1012A00008950F93083090F0982F872F762F652F91
:1012B000542F432F322F22270850F4CF220F331FF1
:1012C000441F551F661F771F881F991F0A95B2F785
:1012D0000F9108952A0D3B1D4C1D5D1D6E1D7F1D38
:1012E000801F911F08950024A7FD00942A17300540
:1012F0004005500560057005800590050895FB01C7
:10130000DC014150504030F08D910190801919F46A
:101310000020B9F7881B990B0895FB01DC014150AF
:10132000504048F001900D920020C9F701C01D9275
:1013300041505040E0F70895E199FECF9FBB8EBB2E
:10134000E09A99278DB30895A8E1B0E042E050E01B
:1013500013C0262FE199FECF1CBA9FBB8EBB2DBBBD
:101360000FB6F894E29AE19A0FBE01960895F1DF64
:10137000272FF0CFDC01CB01FC01E199FECF06C0A5
:10138000FFBBEEBBE09A31960DB20D92415050403A
:08139000B8F70895F894FFCFAF
:101398000001010101010101010101010101010136
:1013A8000101010202020202020202020202020218
:1013B8000202020202020202020202030303030300
:1013C80003030303030303030303040404040404DF
:1013D80004040404040405050505050505050506BA
:1013E8000606060606060607070707070708080889
:1013F80008080809090909090A0A0A0A0A0B0B0B4D
:101408000B0C0C0C0C0D0D0D0E0E0E0E0F0F0F10FD
:101418001010111112121213131414151515161693
:101428001717181819191A1B1B1C1C1D1E1E1F2004
:101438002021222323242526272728292A2B2C2D3F
:101448002E2F3031323334353738393A3B3D3E3F31
:101458004142444547484A4C4D4F51525456585AB8
:101468005C5E60626466696B6D707275777A7C7FAA
:101478008285888B8E9194979B9EA2A5A9ACB0B4C7
:10148800B8BCC0C4C9CDD2D6DBE0E5EAEFF4FAFFB8
:10149800494D524200494D535600494D454D00496A
:1014A8004D425000494D505700494D465200494D54
:0414B800504A000096
:00000001FF
